S00C00006D61696E2E7372656373
S11300000C942A000C9445000C9445000C94450073
S11300100C9445000C9445000C9445000C94450048
S11300200C9445000C9445000C9445000C940B0270
S11300300C9445000C9445000C9445000C94450028
S11300400C9477020C9445000C9445000C944500E4
S11300500C94450011241FBECFE5D8E0DEBFCDBF10
S113006010E0A0E6B0E0E2EFF6E002C005900D92E9
S1130070A036B107D9F710E0A0E6B0E001C01D92A8
S1130080AD38B107E1F70C949E020C940000982F50
S11300908823D4F085958595859580937A00209161
S11300A0640030916500287F3770892F992787FD78
S11300B0909587709070282B392B3093650020938E
S11300C0640020E030E0A5C1209164003091650017
S11300D027703070992787FD90958F779070880FDF
S11300E0991F880F991F880F991F282B392B30933C
S11300F065002093640080917A00843009F4B7C0CD
S1130100853058F48130E9F08130B0F0823009F460
S11301104BC0833009F07BC17BC0863009F4E3C057
S1130120863008F4C4C0873009F401C18F3009F067
S11301306EC121E030E06DC110928A0020E030E011
S113014068C140918A0060E070E0423010F461E0E0
S113015070E020E030E0423011F421E030E080E053
S113016090E0433011F481E090E0822B932B862BB6
S1130170972B892B19F420E030E011C0842F9927A4
S11301809C01220F331F22953295307F3227207F26
S113019032272070877090709068282B392B842F19
S11301A08F5F80938A0035C12115310531F481E0D8
S11301B08093860020E030E02CC12130310531F4F9
S11301C081E08093870020E030E023C122303105B4
S11301D031F481E08093880020E030E01AC12330BC
S11301E0310531F481E08093890020E030E011C1D1
S11301F02050314009F00BC181E080938600809348
S11302008700809388008093890020E030E001C15A
S11302102115310529F41092860020E030E0F9C060
S11302202130310529F41092870020E030E0F1C03C
S11302302230310529F41092880020E030E0E9C032
S11302402330310529F41092890020E030E0E1C028
S11302502050314009F0DBC01092860010928700D4
S1130260109288001092890020E030E0D2C0809182
S11302708600882319F081E08093660080918700CE
S1130280882319F081E08093670080918800882397
S113029019F081E08093680080918900882309F433
S11302A0B6C081E08093690020E030E0B2C0809164
S11302B08600882311F010926600809187008823BD
S11302C011F01092670080918800882311F0109239
S11302D0680080918900882309F499C0109269000C
S11302E020E030E096C080918600882321F030938E
S11302F07E0020937D0080918700882321F0309335
S1130300800020937F0080918800882321F030931F
S113031082002093810080918900882309F477C0AA
S1130320309384002093830020E030E072C08091F9
S113033086008823C1F020916A0030916B0080917F
S11303406A0090916B00220F331F22953295307F03
S11303503227207F322720708770907088609068E1
S1130360282B392B56C0809187008823C1F0209117
S11303706E0030916F0080916E0090916F00220F9B
S1130380331F22953295307F3227207F3227207009
S11303908770907088609068282B392B3AC08091C0
S11303A088008823C1F020917200309173008091FD
S11303B0720090917300220F331F22953295307F83
S11303C03227207F32272070877090708860906871
S11303D0282B392B1EC0809189008823C1F02091DD
S11303E07600309177008091760090917700220F0B
S11303F0331F22953295307F3227207F3227207099
S11304008770907088609068282B392B02C020E098
S113041030E0C90108951F920F920FB60F92112474
S11304208F939F9380917B00982F9F5F90937B0085
S1130430992301F58091850080936000809161008B
S113044080937C00809162008093630080918B0094
S113045080938C00809166008111C09A809167001E
S11304608111C19A809168008111C29A80916900BA
S11304708111C39A80916000981709F4C098809103
S11304807C00981709F4C19880916300981709F4C7
S1130490C29880918C00981709F4C3989F918F910A
S11304A00F900FBE0F901F90189581E083BF89B7FE
S11304B0816089BF08958CEC86B980E090E02AE6DB
S11304C030E0FC01EE0FFF1FE20FF31F11821082D8
S11304D0019688309105A9F70895FC01E770F07042
S11304E0EE0FFF1FE659FF4F8081918108951F92FF
S11304F00F920FB60F9211242F933F938F939F93D4
S1130500EF93FF9387B199278770907024B135B129
S1130510FC01EE0FFF1FE659FF4F31832083019644
S1130520877087B9369AFF91EF919F918F913F9190
S11305302F910F900FBE0F901F901895CFE5D8E024
S1130540DEBFCDBF1ABA8FEF87BB14BA80E481BB7C
S113055010928500109261001092620010928B003C
S113056087E690E00E9440030E945B020E945502CD
S11305701092660010926700109268001092690051
S113058078945F9B04C00E9449030E944700209115
S11305906C0030916D0080917D0090917E00821BF3
S11305A0930B9C0122F422273327281B390B2F3F5E
S11305B0310519F014F02FEF30E020938500181660
S11305C0190614F4C49A01C0C498209170003091A3
S11305D0710080917F0090918000821B930B9C019D
S11305E022F422273327281B390B2F3F310519F01A
S11305F014F02FEF30E0209361001816190614F45C
S1130600C59A01C0C59820917400309175008091FD
S1130610810090918200821B930B9C0122F422277B
S11306203327281B390B2F3F310519F014F02FEF16
S113063030E0209362001816190614F4C69A01C01B
S1130640C698209178003091790080918300909130
S11306508400821B930B9C0122F422273327281B3E
S1130660390B2F3F310519F014F02FEF30E02093B0
S11306708B001816190614F4C79A83CFC79881CF34
S1130680292F332720BD89B988E18AB98EE880BD36
S113069008955F9BFECF8CB1992708955D9BFECF93
S11306A08CB908951F93282F982F92959F70892FA6
S11306B0805D8A3308F0895F922F9F70192F105D37
S11306C01A3308F0195F0E944E03812F0E944E03D3
S11306D01F910895CF93DF93EC018881882331F033
S11306E00E944E03219688818823D1F7DF91CF9110
S10506F0089567
S9030000FC
